:020000040000FA
:0600000093EF06F0120070
:06002A000100460D00007C
:08003000800000000300000045
:0800380004011051600BE842C5
:10004000E842E842E842E842000901E055D0115197
:10005000070A51E00B0A4FE0070A40E0010A2CE0D2
:100060000B0A28E0020A26E0030A22E0080A12E04E
:10007000010A0EE00F0A0AE0030A01E03CD0000189
:10008000010E6B6F0001040E796F36D036D834D074
:1000900090D832D00001010E6B6F00017B0E6C6FA7
:1000A000000E6D6F00017A930001010E706F24D075
:1000B000A8D822D0F4D820D00001010E6B6F040123
:1000C000145100016C6F6D6B7C0E6C27000E6D235C
:1000D00000017A930001010E706F0ED00001010E35
:1000E0006B6F04011451EA6A7C0FE96E000EEA227C
:1000F00012C4EFFF01D000D01200800E0401105D89
:1001000057E11351030A34E0010A10E0030A01E049
:100110004DD00001010E6B6F0001B00E6C6F0B0E25
:100120006D6F120E0001706F716B40D00001010EF7
:100130006B6F04011251F66EF76AD890F636F736F7
:100140007C0EF6260C0EF7220900F5CF6CF00A00A3
:10015000F5CF6DF0020E0001F76A6C25F66E6D5159
:10016000F7220900F5CF70F00A00F5CF71F01ED02C
:100170000001010E6B6F04011251F66EF76AD89000
:10018000F636F736800EF6260C0EF7220900F5CF6C
:100190006CF00A00F5CF6DF06CC0F6FF6DC0F7FF94
:1001A0000800F5500001706F716B00D000017A8378
:1001B00012000001010E6B6F0F0EE66E710EE66EFF
:1001C0000F0EE66EC3EC05F0E552E552E552010E66
:1001D000E66E7C0EE66E000EE66EC3EC05F0E552B0
:1001E000E552E55212C47BF00401125104E1000112
:1001F000050E796F05D00001060E796F85EC04F0CD
:1002000012000401186B196B040110511F0B020A34
:1002100014E0030A0EE0010A01E033D00001010EF0
:100220006B6F0401188100017AA102D004011883C8
:1002300028D00001010E6B6F24D00001010E6B6FFE
:10024000040114510F0B080DF350036A000F026EE6
:10025000040E03221451800B01E0010E040DF35033
:10026000000102246E6F000E03206F6F6EC0E9FF65
:100270006FC0EAFFEF50040B03E00401010E186F9A
:1002800000D000016B050AE10001180E6C6F040E2E
:100290006D6F00017A930001020E706F120004016D
:1002A000120510E110511F0B00090CE10001010EB5
:1002B0006B6F030E0401115D03E100017A8102D02E
:1002C00000017A91040112513AE110511F0B02080A
:1002D00036E114510F0B000932E00001010E6B6F83
:1002E000040114510F0B080DF350036A000F026E46
:1002F000040E03221451800B01E0010E040DF35093
:10030000000102246E6F000E03206F6F030E0401C4
:10031000115D07E1840E6EC0E9FF6FC0EAFFEF6E6A
:100320000ED014AF06D06EC0E9FF6FC0EAFFEF6ACF
:1003300006D0880E6EC0E9FF6FC0EAFFEF6E1200B4
:100340006C5002E0000E01D0010E00090BE0040128
:1003500000513C0BE842E8420D0802E10CD801D004
:1003600040D808D06C5002E0000E01D0010E040904
:1003700001E047D81200D9CFE6FFE1CFD9FFE6521E
:1003800000016A6B6B6B706B716B1CEC00F0DF6AC9
:10039000DF50026E036A010E025C000E03581BE27E
:1003A00000016B5101E017D0F76ADF34FE0BF7361E
:1003B000F66E860EF6260C0EF7220900F5CF02F037
:1003C0000800F5CF03F004D003C0FAFF0250F96E25
:1003D000FBDFDF2ADDD7D5D8E552E552E7CFD9FFDD
:1003E0001200020E00016A5D0AE192D8040100BD0C
:1003F00003D0C80E006F02D0880E006F01D007D95D
:100400001200040E0001795D0AE112C46EFF6E5005
:10041000000803E2050E796F02D0030E796F000128
:100420006A050AE10BD8040104BD03D0C80E046FAD
:1004300002D0880E046F01D0EAD81200D9CFE6FFAF
:10044000E1CFD9FF020EE1260001080E705D000E1B
:10045000715905E270C0DEFF71C0DDFF03D0080EE8
:10046000DE6EDD6A040104930491010EDB50041377
:10047000DFCF05F4000EDB500001705F010EDB5092
:10048000715B180E6E6F040E6F6F00017AA31ED0A1
:10049000D9CFE9FFDACFEAFFEE50ED1016E06CC0DD
:1004A000F6FF6DC0F7FF0800F5506EC0E9FF6FC0A2
:1004B000EAFFEF6E00016E2B000E6F236C2B6D2395
:1004C000DF06010E01E2DB06E3D71CD0D9CFE9FF3E
:1004D000DACFEAFFEE50ED1015E06CC0E9FF6DC019
:1004E000EAFFEF506EC0E9FF6FC0EAFFEF6E000158
:1004F0006E2B000E6F236C2B6D23DF06010E01E2C5
:10050000DB06E4D7D9CFE1FFE552E7CFD9FF1200F0
:10051000D9CFE6FFE1CFD9FF020EE126030E040199
:100520000015E76E010EE7CFDBFF01C4DFFFDE50F1
:1005300000017027DD507123180E6C6F040E6D6F73
:10054000D9CFE9FFDACFEAFFEE50ED1014E06CC02E
:10055000E9FF6DC0EAFFEF506EC0E9FF6FC0EAFF30
:10056000EF6E6E2B000E6F236C2B6D23DF06010EDA
:1005700001E2DB06E5D7D9CFE1FFE552E7CFD9FFAE
:10058000120000016B510CE10401080E016F100E06
:10059000026F040E036F840E006F0401046F35D0E8
:1005A000040110AF22D0000170510401165D00015A
:1005B00071510401175904E216C470F017C471F0A8
:1005C0003DDF0001010E6A6F0401080E016F100E7D
:1005D000026F040E036F800E006F0401180E066F89
:1005E000040E076FC80E046F10D00001020E6A6F70
:1005F0000401056BC80E046F0401080E016F180E8C
:10060000026F040E036FC80E006F6D981200000198
:100610006A6B0401080E016F100E026F040E036F67
:0A062000880E006F0401046B120045
:06062A00F00E8A16931683
:100630009388938A8150100B01E0010E0001726FC4
:100640008150200B01E0010E736F766B776B786B36
:10065000796B010E746F12004BD8060E0001795DA4
:1006600003E36D50020B01E00BD09DD8000907E0B9
:100670000001745102E0000E01D0010E746F01D828
:100680001200000174051EE175510E081AE2766B26
:10069000070E00018015F76A3E0FF66E0D0EF72269
:1006A0000800F5CF77F0020E8025070BF76A3E0FA2
:1006B000F66E0D0EF7220800F5CF78F0802B0001C2
:1006C000756B05D0786B78C077F078C076F0040150
:1006D0000CBF0DD0030EE66E760EE66E000EE66ED3
:1006E0009AEC04F0E552E552E5520001752B120038
:1006F00000018151821104E1100E816F270E826F7B
:100700008107000E825B6DA20BD08151821107E13F
:100710008A708A50010B02E08A8201D08A922FD01F
:100720000001795103E18A908A9229D0790503E189
:100730008A808A8224D0020E795D03E18A808A92BF
:100740001ED0030E795D03E18A908A8218D0050ECF
:10075000795D07E100018151821102E18A708A729C
:100760000ED0060E795D0BE100018151821107E187
:100770008A708A50010B02E08A9201D08A821200AC
:100780008150100B01E0010E0001725D09E0815003
:10079000100B01E0010E726F81B802D0010E02D081
:1007A000000E00D012008150200B01E0010E00016C
:1007B000735D09E08150200B01E0010E736F81BA77
:0C07C00002D0010E02D0000E00D012008A
:0407CC00D38AD38871
:1007D00005D80FD82CEC03F0FCD712000F0EC11275
:1007E0006F6A0001796B00017A6B00017B6B15EF7A
:1007F00003F015EC05F06FBE02D034EC05F01200EA
:0608000093EF06F0120068
:0A080600040110511F0B010801E06E
:1008100079D0145101E076D0060E115D2EE113510E
:10082000230A28E0010A13E0030A01E024D00001B2
:10083000020E6B6F00017B0505E10001D40E6C6FA9
:100840000B0E6D6F090E0001706F716B14D00001FB
:10085000020E6B6F00017B0505E100014A0E6C6F13
:100860000C0E6D6F00017B0504E1320E0001706F0C
:10087000716B01D000D000017A8304011051600B2C
:10088000E842E842E842E842E842010801E03AD0A2
:1008900011510B0A31E0080A21E0090A19E0080A9F
:1008A00009E00B0A05E0080A01E02CD02CD82AD078
:1008B0002BD828D00001020E6B6F00017D0E6C6FEB
:1008C000000E6D6F00017A930001010E706F1AD057
:1008D0000001020E6B6F13C47DF014D00001020EF4
:1008E0006B6F00017E0E6C6F000E6D6F00017A93CE
:1008F0000001010E706F06D00001020E6B6F12C472
:100900007EF000D012001200120000017F6B1E0E5C
:10091000716E0401030E096F200E0A6F040E0B6F37
:10092000880E086F0401230E0E6F040E0F6F400E29
:100930000C6F1200D9CFE6FFE1CFD9FFE652FC0ED3
:10094000DB50030805E2030EF36EFC0EF3CFDBFF72
:10095000DF6AFC0EDB50DF5C19E2DF50E76EFD0E54
:10096000DBCFE9FFFE0EDBCFEAFFE750E926000E02
:10097000EA22EF50E66EDF50EA6A230FE96E040EBA
:10098000EA22E552E750EF6EDF2AE3D7FC0EDBCF19
:100990000DF4400E04010C170C7D880E0C13E5526B
:1009A000E552E7CFD9FF1200D9CFE6FFE1CFD9FF5B
:1009B00000017F6B040108BF31D0FC0EDBCF02F0D9
:1009C0000951D880025403E2FC0E09C4DBFF000188
:1009D0007F6BFC0EDB507F5D19E27F51EA6A200FCE
:1009E000E96E040EEA22EF50E66E7F51E76EFD0ECF
:1009F000DBCFE9FFFE0EDBCFEAFFE750E926000E72
:100A0000EA22E552E750EF6E7F2BE3D70401030E95
:100A1000096F400E0817087D880E081300017F51EA
:0A0A200000D0E552E7CFD9FF120025
:060A2A006DA60FD802D0FA
:100A30006DB613D80001790508E16DBA06D0686A71
:100A4000696A69806988020E796F12006D6A696A45
:100A50006D860001010E796F12006D6A696A0001EE
:100A6000796B12002DEF05F00001795101E13AD0C8
:100A70006850040B04E06950040B01E041D86DB2EA
:100A800031D06850010B04E06950010B01E059D8E6
:100A90006850100B04E06950100B01E024D8685036
:100AA000400B04E06950400B01E040D86850200B37
:100AB00004E06950200B01E03BD86850020B04E0D1
:100AC0006950020B01E03BD8030E0001795D01E2A1
:100AD00009D06850080B06E06950080B03E0A0EC51
:100AE00001F068961200698468986D82A19AF2906C
:100AF000A08AF2860300F2B007D8A09AF2961200FC
:100B00006D9269946894120000017AA10ED0F8DF0A
:100B10006D840001080E836F070E846F8307000E3B
:100B2000845B83518411FAE16D941200689C120079
:100B300070A003D007EC03F07090689A12006892DE
:100B400012006A6A686A9F0E6B6E7B0E696E6E6A2F
:100B50000F0EE66E710EE66E0F0EE66E14D8E552BD
:100B6000E552E552160E706E68A602D06896FCD764
:100B70006D9807EC03F000017A9100017B6B000196
:100B8000030E796F1200D9CFE6FFE1CFD9FFFD0E3A
:100B9000DBCFE9FFFE0EDBCFEAFFFC0EDB5004E00B
:100BA000EE6AFC0EDB06F9D7E552E7CFD9FF12005B
:100BB0001201000200000008D80400000100010238
:100BC000000109022200010100A032090400000115
:100BD0000301020009210101000122320007058101
:100BE0000303000A0403090434034D006900630091
:100BF00072006F00630068006900700020005400FC
:100C00006500630068006E006F006C006F00670095
:100C10007900200049006E0063002E002E034D0075
:100C20006F00750073006500200049006E00200011
:100C30006100200043006900720063006C006500E1
:100C40002000440065006D006F0005010902A1014C
:100C50000901A100050919012903150025019503C2
:100C60007501810295017505810105010930093180
:100C70001581257F750895028106C0C0C20BC20B85
:080C8000E40BE80B1C0C060854
:080C88002A0EF66E000EF76E55
:100C9000000EF86E00010900F550656F0900F5506F
:100CA000666F03E1656701D03DD00900F550606FC4
:100CB0000900F550616F0900F550626F09000900E5
:100CC000F550E96E0900F550EA6E090009000900C7
:100CD000F550636F0900F550646F09000900F6CF05
:100CE00067F0F7CF68F0F8CF69F060C0F6FF61C039
:100CF000F7FF62C0F8FF0001635302E1645307E0AD
:100D00000900F550EE6E6307F8E26407F9D767C093
:100D1000F6FF68C0F7FF69C0F8FF00016507000E25
:060D2000665BBFD7120064
:0A0D260013EE00F023EE00F0F86A6F
:0E0D3000019C44EC06F0E6EC03F0FDD7120047
:020D3E00FCFCBB
:060D4000FC0004040400A5
:030D4600000000AA
:020000040030CA
:0E000000100F3F1E008181000FC00FE00F4067
:00000001FF
